:020000040800F2
:101400000020002011160008B94E0008BB4E00084D
:10141000BD4E0008BF4E0008C14E0008000000008D
:10142000000000000000000000000000C34E0008A3
:10143000C54E000800000000C74E0008C94E000855
:10144000591600085916000859160008854F00085B
:101450005916000859160008E54F00089D4F00086E
:1014600059160008591600085916000859160008A0
:101470005916000859160008591600085916000890
:1014800059160008591600087550000800000000A1
:1014900000000000000000000000000059160008D5
:1014A0005916000859160008591600085916000860
:1014B0005916000859160008591600085916000850
:1014C0005916000859160008591600085916000840
:1014D00059160008A15000085916000859160008AE
:1014E0005916000859160008591600080000000097
:1014F00000000000000000000000000000000000EC
:1015000000000000000000000000000000000000DB
:1015100000000000000000005916000859160008DD
:1015200000000000000000000000000000000000BB
:1015300000000000000000000000000000000000AB
:10154000000000000000000000000000000000009B
:10155000000000000000000000000000000000008B
:10156000000000000000000000000000000000007B
:10157000000000000000000000000000000000006B
:10158000000000000000000000000000000000005B
:10159000000000000000000000000000000000004B
:1015A000000000000000000000000000000000003B
:1015B000000000000000000000000000000000002B
:1015C0000000000000000000000000005FF808F1CB
:1015D00010B5054C237833B9044B13B10448AFF36D
:1015E00000800123237010BD1C00002000000000BB
:1015F000545D000808B5034B1BB103490348AFF322
:10160000008008BD0000000020000020545D00089C
:10161000002103E00B4B5B58435004310A480B4B4D
:1016200042189A42F6D30A4A02E0002342F8043BE9
:10163000084B9A42F9D303F0CBFD03F075FE01F09D
:10164000BFF9FEE7745D0008000000201C000020C8
:101650001C00002068020020FEE7000040F0BF6090
:10166000024B40F40030D860704700BF00ED00E04E
:10167000C27810B503780AB3164A03F16043D16803
:101680004278C943C1F30221C1F1040402FA04F40F
:101690000F22CA40817803F561430A4022431201B8
:1016A000D2B283F8002303780122590903F01F0303
:1016B00002FA03F3084A42F8213010BD5A09012109
:1016C00003F01F0301FA03F30349203241F82230EB
:1016D00010BD00BF00ED00E000E100E0044B042875
:1016E0001A680CBF42F0040222F004021A6070472C
:1016F00010E000E0436810B523F470220B6822F478
:10170000807213430A7943EA02234360CA688B68F4
:1017100084681A43084B234013434A7943EA42033F
:101720008360C36A23F470020B7C013BDBB242EAA4
:101730000353C36210BD00BFFDF7F1FF836811B111
:1017400043F0010301E023F00103836070478368E5
:1017500011B143F4807301E023F480738360704718
:10176000C9B243680AB1194301E023EA01014160AB
:101770007047836843F00803836070478068C0F354
:10178000C0007047836843F004038360704780683B
:10179000C0F380007047836811B143F4A00301E0F7
:1017A00023F4A003836070478068C0F380507047C3
:1017B000092970B50DD9A1F10A04C66804EB4404E7
:1017C0000725A54026EA050503FA04F42C43C46066
:1017D0000AE0066901EB41040725A54026EA050554
:1017E00003FA04F42C430461062A0CD8013A446B32
:1017F00002EB82021F23934024EA030301FA02F260
:101800001A43426370BD0C2A0CD8073A046B02EBF2
:1018100082021F23934024EA030301FA02F21A43CF
:10182000026370BD0D3AC46A02EB82021F2393402B
:1018300024EA030301FA02F21A43C26270BD0000F7
:10184000044B9A6810B142F4000201E022F4000255
:101850009A60704700240140C943016070476FEAF5
:10186000112101607047000082B000230193044BF6
:101870000193019B18440190019B196002B07047CD
:10188000006C004082B000230193054B0193019B43
:1018900018440190019B188880B202B0704700BFC5
:1018A000006C00404FF6FE73026813400360002393
:1018B000036043608360C360284B984201D1284A8B
:1018C00027E0284B984201D1254A2AE0264B98422E
:1018D00001D1234A2DE0254B984201D1204A30E026
:1018E000234B984201D11E4A33E0224B984204D147
:1018F0001B4A536843F470032EE01F4B984204D1F7
:10190000174A536843F0706326E01C4B984204D199
:101910001B4A536843F00F031EE01A4B984204D150
:10192000174A536843F0F00316E0174B984204D16E
:10193000134A536843F470630EE0144B984204D189
:101940000F4A536843F4704306E0114B984204D1A8
:101950000B4A536843F470235360704708000240F9
:10196000000002401C0002403000024044000240DF
:10197000580002406C00024080000240080402400F
:10198000000402401C0402403004024044040240AF
:10199000580402400A6A10B58C68036814430A6947
:1019A00023F4FF4314434A6923F0700314438A6904
:1019B0001443CA6914434A6A14438A6A224313438C
:1019C0000360CB6843600B6883604B68C36010BDE5
:1019D00019B1036843F0010303E04FF6FE73026898
:1019E0001340036070470000044B00221A605A60E5
:1019F0009A60DA60024A5A61704700BF00040140F1
:101A0000FFFF0F00827970B50168037942B3CE43BE
:101A1000184A03F18043156803F582333540156099
:101A20005468344054601C6821431960016894680C
:101A3000CD432C409460D3682B40D3604379102B66
:101A400006D193680B439360D3681943D16070BD8E
:101A500003F1804303F582331A681143196070BDA6
:101A600003F1804303F582331A6822EA01021A6007
:101A700070BD00BF00040140054B1A685B6903405C
:101A800004D0024214BF012000207047184670475E
:101A900000040140014B5861704700BF0004014041
:101AA000034B044A5A6002F188325A60704700BF03
:101AB0000020024023016745FFF7F2BF024A136985
:101AC00043F080031361704700200240FFF7F6BF28
:101AD000014BD860704700BF00200240084BDA6815
:101AE000D10709D4DA68520708D4DB6813F0100F65
:101AF00014BF032004207047012070470220704764
:101B00000020024010B50446FFF7E8FF012806D187
:101B10001CB1FFF7E3FF013CF8E7052010BD002CE6
:101B200008BF052010BD000070B505464FF40050F9
:101B30000E46FFF7E7FF04280ED1084C4FF4005083
:101B4000236943F0010323612E80FFF7DBFF41F699
:101B5000FE7322691340236170BD00BF0020024064
:101B600038B505464FF43020FFF7CCFF042812D1DA
:101B7000094C4FF43020236943F00203236165616F
:101B8000236943F040032361FFF7BCFF41F6FD7377
:101B900022691340236138BD00200240014B1860C8
:101BA000704700BF00300040014B5860704700BFD5
:101BB00000300040014B9860704700BF003000408B
:101BC0004AF6AA22014B1A60704700BF003000405D
:101BD0004CF6CC42014B1A60704700BF0030004009
:101BE000064B002201281A701A7002D0042802D075
:101BF00070471870704705221A7070472010024015
:101C0000024A136A18431062704700BF0010024076
:101C1000014B1860704700BF3C0442421E4A10B599
:101C2000536803F00C03042B03D0082B03D01B4B89
:101C300012E01B4B10E053685168C3F38343C903A0
:101C400041BFD16A164C01F00F0101314CBFB4FB0A
:101C5000F1F1144902334B4303605368124CC3F350
:101C60000313E15C0368CB4043605168C1F3022178
:101C7000615C23FA01F181605168C1F3C221615CAA
:101C8000CB40C36052680949C2F381328A5CB3FB1E
:101C9000F2F3036110BD00BF0010024000127A0091
:101CA000808D5B0000093D00040000200000002042
:101CB000044B5A6909B1104301E022EA000058615F
:101CC000704700BF00100240044B9A6909B11043ED
:101CD00001E022EA00009861704700BF0010024056
:101CE000044BDA6909B1104301E022EA0000D8612F
:101CF000704700BF00100240014B1870704700BFD2
:101D0000071002404209012A074B01D11B6803E07A
:101D1000022A0CBF1B6A5B6A00F01F0023FA00F066
:101D200000F00100704700BF00100240034A938892
:101D30009BB243F010039380704700BF002800401F
:101D4000034A938823F010031B041B0C93807047F5
:101D500000280040034A938B108B9BB243EA00405B
:101D6000704700BF0028004008B5FFF7DFFF044BB5
:101D7000020C80B21A839883BDE80840FFF7E0BFE9
:101D80000028004008B5FFF7D1FF054BC0F3034220
:101D900080B21A819881BDE80840FFF7D1BF00BF2B
:101DA00000280040064B9A881B8892B2034005D059
:101DB0001040C0B2003018BF01207047184670476D
:101DC00000280040034A93889BB223EA00009080D9
:101DD000704700BF0028004070B50E460446038AD5
:101DE000CA889BB223F440531343038282898988B3
:101DF000338992B20B43718922F4B0520B4322F023
:101E00000C0213439BB28381838AB2899BB223F471
:101E1000407386B01343838201A8FFF7FFFE174A81
:101E2000039B049D3168944218BF1D4619226A43E2
:101E3000A389642613F4004F14BF4D008D00B2FB3C
:101E4000F5F5B5FBF6F0A28900010109120406FBC5
:101E5000115307D5D9003231B1FBF6F202F0070277
:101E6000104306E01A013232B2FBF6F303F00F031F
:101E7000184380B2208106B070BD00BF0038014019
:101E8000838919B19BB243F4005303E023F4005358
:101E90001B041B0C83817047012310B5C1F342144E
:101EA0009C4201F01F0103FA01F101D10C3003E063
:101EB000022C0CBF1030143003680AB1194301E042
:101EC00023EA0101016010BDC1F308018180704760
:101ED0008088C0F308007047012310B5C1F3421495
:101EE00001F01F029C4203FA02F201D1838903E050
:101EF000022C0CBF038A838A9BB21340028892B2E1
:101F000043B10123090A03FA01F10A4214BF18463A
:101F1000002010BD184610BD0E4B4FF080625A6075
:101F20000D4911229A600022C3F80C28C3F8041846
:101F30000A49C3F80018C3F80C2C4FF03332C3F829
:101F4000042C02F1885202F580121132C3F8002CE1
:101F5000704700BF00000140BB34333303004033FF
:101F600008B50620FFF7C8FE00214FF48040FFF7B8
:101F7000ABFE012144F20D20FFF7A6FE01214FF038
:101F80000050FFF7ADFEBDE8084001210846FFF70D
:101F90008FBE000007B54FF4C060FFF75FFB1D4B1D
:101FA00001A8DA68C2F30222C2F10703111D042B53
:101FB00028BF042306294FF0010101FA03F303F1BE
:101FC000FF338CBF033A00220B4093401B01114AA0
:101FD000DBB282F8233025238DF8043000238DF8FE
:101FE00007108DF80630FFF743FB122301A88DF888
:101FF0000430FFF73DFB062301A88DF80430FFF7FE
:1020000037FB072301A88DF80430FFF731FB03B03D
:102010005DF804FB00ED00E008B56FF00400FFF789
:102020005DFB45F6BF52054BF0215A60044A82F829
:10203000231000229A6007221A6008BD10E000E019
:1020400000ED00E007B5FFF7CFFC002201238DF87B
:1020500004206846082200938DF805208DF806308C
:10206000FFF7D0FC022368460093FFF7CBFC03B0D8
:102070005DF804FB1FB5104C4FF41653009300237A
:10208000ADF80430ADF80630ADF80830ADF80C30DE
:1020900069460C232046ADF80A30FFF79DFE012269
:1020A000204640F22551FFF7F7FE01212046FFF7B9
:1020B000E7FE04B010BD00BF0038014070B53748DE
:1020C00090B0FFF7EFFB364B00250593354B042608
:1020D000069380230A934FF480730B934FF480632D
:1020E0000C9320230D9305A94FF400532B480E9316
:1020F0000795089609950F95FFF74CFC0121274895
:10210000FFF766FC01244FF46023694626480293DA
:1021100000958DF804408DF8055003958DF81060FA
:10212000FFF7E8FA0523224621461F48FFF740FB48
:102130000222114605231C48FFF73AFB0523032220
:1021400010211948FFF734FB0523324603211648B6
:10215000FFF72EFB2046FFF773FB22464FF4087172
:102160001148FFF7FDFA21460F48FFF7F0FA0E4835
:102170002146FFF7E3FA0C48FFF7FBFA0A48FFF79E
:10218000FDFA0028FAD10848FFF7FCFA0648FFF7E5
:10219000FEFA0028FAD110B070BD00BF080002405E
:1021A0004C240140100200200024014008B545F2F3
:1021B0005550FFF7F3FC0520FFF7F6FC7D20FFF7F5
:1021C000F9FCFFF7FDFCBDE80840FFF701BD00008A
:1021D00070B5294C012126464FF0C050FFF780FD15
:1021E000264A01201368264D43F4837343F001030C
:1021F0001360244A136943F004031361FFF7F0FCF2
:10220000002323604120FFF77DFD28B92368AB42FE
:1022100002D801333360F5E72268194B9A4229D876
:102220004FF48070FFF7ECFC0120FFF7F1FC16493A
:10223000114A8B88154823F008031B041B0C8B8064
:10224000002313601A468D882D0705D563B10C4B0A
:1022500022609A420ED807E0824202D00132012366
:10226000F1E70BB1226070BD47F6FF70BDE870402A
:10227000FFF788BD70BD00BFB000002000700040B7
:1022800097801E0000ED00E00028004098801E00AE
:10229000024B0001012298605A60704700740040B0
:1022A000074B9B8A0341DB0709D5064AD36823F015
:1022B0004003D360044B01221A70044B187070471E
:1022C0002402002000080140EC00002058020020F9
:1022D0004FF6FF70F0B50A23642101FB03F202F10F
:1022E0000062B2F89C2F824202D1013BF5D101235A
:1022F000322058432A4C00228118490001F1006124
:10230000B1F89E3F24F8123001320D2A244BF3D14C
:10231000244C254D254E991D0022171931F8020F26
:102320003F89B84203D897193F89B84202D2501961
:10233000008908800232082AEFD11A68013202BFF0
:10234000174A002111605A68013202BF144A002165
:1023500051601969164A914282BF114A00211161E8
:102360009A8A12F4404F02BF4FF6FF710C4A9182D5
:10237000DA8A1B8B643A92B2B2F5487F88BF084A6A
:10238000A3F164039BB284BF4FF49671D182B3F57D
:10239000487F82BF024B4FF4FA721A83F0BD00BF30
:1023A0002402002088530008745300089C5300083E
:1023B0003F420F004FF6FF712DE9F84364220024DD
:1023C00002FB04F303F1006303F580531B888B4287
:1023D00002D001340A2CF3D1FFF76EFB3520FFF752
:1023E00077FB0A2C05D12B48FFF7BAFB0428FAD15A
:1023F000002464235C4304F1006505F580554AF62A
:1024000055212846FFF790FB0428F8D1224E234F90
:102410000025264406EB050805EB0709B9F800106E
:102420004046FFF781FB0428F8D102351A2DF1D17F
:102430001B4B1C4E1A781C4F12F0800F18BF73787C
:102440004FF000051CBF63F07F037370530648BF55
:102450007378274444BF43F04003737007EB0508CB
:1024600006EB0509B9F800104046FFF75DFB0428AC
:102470000C4CF7D10235482DF0D1637803F03F03BF
:102480006370FFF723FB054B987BBDE8F843FFF72C
:10249000FFBE00BF00100008021000082402002048
:1024A000DF000020EE0000201C100008FFF782BFB4
:1024B000FFF780BF4FF6FF7070B50A23642101FB60
:1024C00003F202F10062B2F89C2F824202D1013B7A
:1024D000F5D1012332221A485343002299184900AA
:1024E00001F10061B1F8B81F20F812100132242A5E
:1024F0001349F3D14B78180604D51248027862F0DC
:102500007F0205E05A0604D50E48027842F04002E8
:10251000027003F03F030C480C4C4B70002303F097
:10252000030231F8136030F81250AE4284BF34F821
:10253000122021F813200133242BF0D170BD00BFED
:10254000EE000020DF000020B8530008B053000860
:10255000254B1B88B3F5FA7F30D340F24D229342CE
:102560002ED940F29D2293422CD940F2ED22934283
:102570002AD940F23D32934228D9B3F5617F27D35F
:1025800040F2C932934225D9B3F57F7F24D340F27C
:102590002D42934222D9B3F58C6F21D3B3F5916FBD
:1025A00020D3B3F5966F34BF0B230C230F4A116869
:1025B0001944116051680B44536070470023F5E7DC
:1025C0000123F3E70223F1E70323EFE70423EDE719
:1025D0000523EBE70623E9E70723E7E70823E5E719
:1025E0000923E3E70A23E1E7A600002024020020F4
:1025F000174938B50B883E2203EB8303B3FBF2F394
:10260000144A9BB214890846A3421146124A88BF55
:102610001B1B138040F6E443408849894343C3F3BE
:102620000F338B420D4D10D95B1A0A499BB28C892E
:10263000108863434324B3FBF4F402F033FE2044D8
:1026400080B202F03BFE288038BD13882B8038BD55
:10265000EC010020240200201C020020C400002005
:1026600010B50F4C3C236078A27843434FF461606F
:1026700000FB023320781844FFF776FB2179A37919
:1026800001F01F0141EA4321637904205B0103F457
:10269000F073194389B2BDE81040FFF7E5B800BFF9
:1026A00000020020054B06495A79022A885C04D1B1
:1026B0009B799B0704BF0130C0B270470002002025
:1026C000C05300082DE9F843FFF744FB324B0546A1
:1026D0009842324E3CD9324C3746B0FBF4F4337951
:1026E0004FF001081C44A4B24FF00009FFF7DAFFD5
:1026F00080B2844213D97379241A0133DBB20C2BD4
:10270000A4B201D87B71F1E7BB7987F8058001336A
:10271000DBB2632B94BFBB7187F80690E6E7737951
:10272000B1795B01E4B203F4F07343EA41233471FD
:1027300004F01F0444EA0301042089B2FFF794F86F
:10274000174BB5FBF3F203FB12552846FFF70CFBC2
:10275000A9B20820FFF788F80C20FFF793F8EB03E5
:102760004CBF40F0010120F0010189B20C20FFF7BD
:102770007BF84FF46162B5FBF2F3B37002FB1353C5
:102780003C22B3FBF2F37370B5FBF2F302FB13557B
:102790003570BDE8F88300BF7F51010000020020C2
:1027A0008051010070B5204A204B12781C4652001F
:1027B00002F07E011E4A1E1D12781025D20102F47D
:1027C00078620A439A801B4A12789A711A4A1278E0
:1027D000DA711A4A12881A81194A12785A81194AEA
:1027E00012889A81184A1288DA81184A12881A8245
:1027F000174A12885A822846043536F8021FADB2AD
:10280000FFF732F82C2DF6D10C20FFF73BF8A1880A
:1028100000F0010021F00101014389B20C20BDE864
:102820007040FFF721B800BFEC000020CA00002074
:10283000BE0000201F020020FC0100200802002032
:10284000DF0000204A0200203E0100203C01002061
:10285000E6010020F8B5494D04242046FFF712F8A0
:102860000434A4B22C2C25F8020FF6D1444B454871
:102870001A88454C02F01F010171C2F343114171E6
:102880009988520A8271414DC1F34502022A227091
:102890002A701C4607463E4E01D0042A48D165885E
:1028A000CA0748BF45F48035FFF70CFF7A783C2310
:1028B0005343B9784FF4616202FB01323B78134411
:1028C0009D4284BF03F5A83303F5C0730A35AB42BC
:1028D0002AD2A3882F4AC3F3C4131370A2792E4BB4
:1028E000218A1A70E379228933702C4B1A80A37ADB
:1028F0002B4A13709B0641BF2A4A137843F0080302
:102900001370A289284B1A80E389284A1380284A29
:102910001180618A274A1180274A1380FFF7CAFD78
:10292000264B00221A7023E00420FFF7B9FC1FE0B9
:10293000053A012A1AD8174AC1F3C41111709979BE
:10294000154A188A1170DA7919893270134A118080
:102950009989154A1180DA8914490A801449088036
:10296000598A144B1980144B1A8001E000232B70F4
:10297000337803F0BF033370F8BD00BFC8000020F8
:10298000CA0000200002002016000020EC000020F9
:10299000FC010020BE0000201F02002008020020D1
:1029A000DF000020650200204A0200203E010020D6
:1029B0003C010020E601002048020020C800002061
:1029C0002DE9F04F934B944A85B01A60FFF7C8FA8F
:1029D000FFF7FEFBFFF7A0FA904B1B78A82B00D067
:1029E000FEE7FFF7D7FAFFF769FB8D4B1A688D4BAF
:1029F0009A4208D98C4A0D20136A23F0010313620E
:102A0000FFF74EFC10E0894B9B6813F020030BD1BD
:102A100087490A7842F020020A70864A00BF0133D3
:102A20009342FBD1844A1360844C854DE36843F0A4
:102A30004003E360FFF74CFCFFF70CFFEA8A814B91
:102A40001A802A8B804B1A8040F63F327F4B1A60E7
:102A5000A87BFFF71DFCFFF70DFBFFF7F3FAFFF76D
:102A6000A5FBFFF7D9FA714B9B68019413F0800F17
:102A7000774B07D000221A70764F774A32231370B3
:102A80003E4671E00122F6E73B78012B79D1674A97
:102A9000536943F480435361704C237818067AD409
:102AA00023786E4A13F0040FDFF8848140F0AC8184
:102AB00098F80030DFF8A89113F0200F40F002845E
:102AC00099F80030664AD90700F14B842378634AAD
:102AD000DB0707D5137803F0FE031370FFF7F2FD51
:102AE000FFF760FE23785D4A580608D5137803F097
:102AF000BF031370FFF75EFCA87BFFF7C9FB98F8D4
:102B000000304B4A190621D51378564903F07F034C
:102B10001370554BB1F802C05A89B1F800E0624415
:102B200052105A801A898888724452101A809A89E1
:102B3000C988024452109A80DA89A3F80AC00A446C
:102B40005210DA80A3F808E09881D9813378012BFC
:102B500040F01F84454B1B78022B05D93D4B1A785A
:102B6000434B53F822309847FFF72AF8414B1A7825
:102B7000120789D51A7802F0F7021A7000F074FF74
:102B800082E73D4B1B789C0602D500F073FC83E77F
:102B900000F0DEFC80E7237803F07F03237000F071
:102BA000A5FD364B00221A70304A13780133DBB290
:102BB000632B88BF0A231370314A13780133DBB2C9
:102BC000632B88BF0A2313702E4A138801339BB2EC
:102BD000B3F5616F01D813800FE0002313800F4B12
:102BE0001B78A82B00D0FEE7274B1A682B689A4267
:102BF0001EBF237843F0400323703378052B52D156
:102C0000224B1B78042B43D1EB890A2B48D90A3B72
:102C100044E000BF440000204C000020FF0F0008EB
:102C2000B000002097801E0000100240000C014000
:102C3000FC01002020A10700B8000020000801408E
:102C4000240200206202002066020020007400407E
:102C5000E5010020EC00002046020020A800002032
:102C6000C300002010020020EC010020C80000205A
:102C7000D05300081E020020DF0000204002002088
:102C8000E90100204800002002100008BE000020DA
:102C9000052B08D1EB89FD2B02D80133A04AD38143
:102CA000A87BFFF7F5FA237843F001032370FFF7C1
:102CB0004FFC9C4A1378D9074CBF9B499B490B8812
:102CC00001330B8013781B0611D5964B1B785806E1
:102CD0000DD4974B93F90020944B1B8853433C220F
:102CE00093FBF2F3934A12881344934A138096F8A5
:102CF00000E0BEF1010F6BD040F684738F4A90481C
:102D0000518899420CD903780133DBB2092B81BF7A
:102D1000002303708B48037888BF43F0010300E071
:102D200000230370019B9B6813F0200F864B06D095
:102D30008648B0F800C040F22D40844511D9BEF15C
:102D4000050F0ED01B7880480133DBB2092B81BF01
:102D5000002303707B48037888BF43F008030370A7
:102D600001E0002018700B2979490CD80B78013349
:102D7000DBB2092B81BF00230B7072490B7888BF2F
:102D800043F0020300E000230B701288714B0B2A02
:102D90000BD81A780132D2B2092A18D900221A7037
:102DA000684A137843F004030EE0B2F5CD6F0DD9F5
:102DB0001A780132D2B2092A1A7009D900221A707F
:102DC000654A137843F00103137001E000221A7082
:102DD000624A936813F0200F614B08D09268510645
:102DE00003D50320FFF75CFA5AE61A7805E05D4A3E
:102DF000127812F0200F1A7802D042F0200201E07F
:102E000002F0DF021A704BE6137803F0FB03137035
:102E1000554B00221A80554B1B7813B1013B534A86
:102E200007E0534B1B88642B04D9464A137843F0C0
:102E30008003137000F0FEFBFFF7DAFB4D48FEF74E
:102E4000B3FC18B901214B48FEF7A5FC4A484B4B8F
:102E500002881B88DFF83CE11344384ADFF838C1A8
:102E6000D188BEF800209BB20A449CF8001092B2B0
:102E70000131C9B21F290380AEF800208CF8001080
:102E800023D932495B090B80394952090A8098F8E5
:102E90000010DFF8CC9001F0400101F0FF0231B1E9
:102EA000002303808CF80030AEF800300DE099F874
:102EB000001041F0400189F80010314921F812302A
:102EC0000132D2B2062AF9D1EAE72E4B15491B7816
:102ED000DFF8C8A0DFF8C890002B00F0C0812A4AB4
:102EE0002A4813780133DBB2632B01D8137082E0D8
:102EF000322313700B78154A13F0010F14BF244BC3
:102F00000D4BB2F800E01B88CEEB03031BB2322B53
:102F100048DC6FF0310E7345B8BF734643E000BF25
:102F2000240200201F020020380100200802002097
:102F3000400000203E01002048020020EC0100205B
:102F40001A020020E8010020C2000020A600002094
:102F5000A40000200D02002041020020000C0140CE
:102F6000FC010020DF000020420200204602002079
:102F7000E200002000240140AC000020C40000203A
:102F80004C020020C8000020EB010020E0000020DF
:102F90004A02002044020020B6000020EA0100207E
:102FA000AA0000203223B2F800C09BB2CCF5334215
:102FB000E23292B20CF5967C92FBFCF2DFF870B331
:102FC00003EB830E4FEA4E0EA0F800E0BBF800E0E2
:102FD0000EF1010E1FFA8EFE72453FBFDFF814E3BB
:102FE0000022ABF80020BEF800202EBFABF800E0B6
:102FF0009B18AEF80030BB4B1A780132D2B2312A9E
:1030000035D94FF0000C83F800C0B74BDFF8E0B2C1
:10301000B3F800E0B54B1A780FFA8EF33BF912B013
:10302000CBEB030303EB8303DFF808B39B001BB276
:10303000ABF8003091F800B01BF0010FDFF8F8B2E8
:1030400018BF8BF800C09BF900C0C3EB0C0303EB67
:103050008303DFF8A8C25B00ACF80030A44B23F870
:1030600012E00132D2B2052AA04B88BF00221A70AA
:10307000A04AB2F90030642BC4BF64231380B2F9B4
:1030800000306433BEBF4FF69C7E9A4BA3F800E03D
:10309000B0F900301288642BC2BF974B4FF0640E1A
:1030A000A3F800E0B0F900306433BEBF4FF69C7E59
:1030B000914BA3F800E0914B0088B3F900E0104475
:1030C000BEF1640FC4BF4FF0640EA3F800E0B3F983
:1030D00000E01EF1640FBEBF4FF69C7CDFF81CE2DF
:1030E000AEF800C01A8883189BB21AB28448002A2E
:1030F000028014DD642AC8BF64238AF800309AF87D
:103100000020642393FBF2F2D3B2012A7D4AC8BFA8
:1031100043F0010313700B7843F0020305E0002332
:103120008AF800300B7803F0FD030B7098F800303C
:103130009A0603D5019B9B689B0603D40B7803F08A
:10314000FD030B70DFF8F4B19BF800300133DBB204
:10315000632B8BF8003030D96B4B4FF0000C83F8A9
:1031600000C0684B8BF800C01A78684B1A70684B27
:10317000684A187892F800E01D308645DFF8C0E113
:1031800016DD9EF800000130C0B2052802D88EF886
:1031900000000FE00C20039202938EF800C0FFF7AE
:1031A0007FF80878029B00F0FD000870039A01E0A8
:1031B0008EF800C00020107018700B78980752D558
:1031C000554B1B781A064ED54E4B93F800E0BEF1D6
:1031D000040F22D94D489BF800300278DFF828C14F
:1031E000934203D09CF80030DB073CD59CF80030BC
:1031F00013F0010F04BF724402703278012A37D0F5
:10320000B9F8002043480132A9F8002002780133C0
:10321000013202708CF8003013E09BF800309AF80D
:1032200000209A4212D99A0710D53378012B1FD06B
:10323000B9F80030374A0233A9F800301378013367
:103240001370364AD36843F4004310E0334AD3681E
:1032500023F40043D360324B00221A7008E00B784D
:1032600003F0FD030B702D4AD36823F40043D360B1
:103270009AF80030612B1CD90B789B0719D54EF6B4
:103280006023B9F800209A427FF612AC254B002249
:103290001A80254A144B1988138803339942D7BFE3
:1032A000224A1180137843F04003D8BF1370FFF710
:1032B000FFBB0023A9F800300B4B1A881A4B1A8069
:1032C000FFF7F6BB99F8003098077FF5F9AB337834
:1032D000012B37D199F8003003F0FD0389F8003055
:1032E000FFF7EEBB20020020A6000020C600002051
:1032F0004C020020E6010020E00000200E02002029
:1033000022020020C100002038000020BC00002064
:103310000C020020C00000201F020020000C014011
:1033200036010020AA00002042000020E801002011
:103330003A0100204201002040000020440100200A
:1033400059020020FFF7BEF9FFF72CFAFFF732F819
:10335000FEF736FC3B78012B3FF4B2AB30BFFFF7F2
:10336000AFBB3378012B05D1137803F0FE03137044
:10337000FFF7ACBBFFF7A6F9FFF714FAFFF71AF84F
:10338000FEF71EFC3B78012B3FF4A0AB30BFFFF7EC
:103390009DBB334B1B780A2B7FF6DCAB2278314B7D
:1033A00012F0200F1A7804D002F0DF021A70002009
:1033B00052E0120705D51A78082002F0F7021A70B9
:1033C0004AE0294A1378D80701D5062044E013784B
:1033D000190706D5254A0520D36823F40043D36096
:1033E0003AE013789B0701D5092035E01378580798
:1033F00001D50A2030E01E4B1B78D90701D50E20DD
:103400002AE01378DB0601D50B2025E02378154947
:10341000D80605D50B78072003F0EF030B701BE0EF
:103420001278114B12F0200F1A7804D002F0DF024C
:103430001A700C2010E012F0400F1A7804D002F03D
:10344000BF021A70012007E012067FF583AB1A78DD
:10345000022002F07F021A70FEF722FFFFF77ABB0C
:10346000E9010020A8000020E8010020000C014034
:103470004102002010B5314B314819780131C9B2F1
:1034800019700378DA0615D52E4A946864060ED4AE
:10349000546944F4005454612B4C2488002C3DD1D1
:1034A000516923F0100341F48041516115E023F08C
:1034B00010033CE09A0615D5224A9468A4060ED45F
:1034C000146944F4005414611F4C248834BB5169BE
:1034D00023F0200341F480415161037010BD23F0BB
:1034E000200324E0DA070BD5164A9468640604D456
:1034F000536943F4005353610CE023F0010316E0D9
:103500009A0719D50F4A9468A4060ED4136943F498
:10351000005313610D4B1B789B0601D57E2907D8FC
:10352000136943F48043136110BD23F00203037059
:10353000536943F48043536110BD00BF5A02002019
:1035400065020020000C014018000020DF00002070
:1035500010B53349334A0B78084613F0010F20D0D9
:103560009168490604D4536943F40053536121E040
:1035700023F001010170516941F4804151615A0702
:103580004DD529490A780132D2B2C82A84BF23F026
:103590000503037003780A7043F0020303700F22DF
:1035A00031E09C0724D59068800608D4136943F461
:1035B00000531361136943F48043136110BD03F09A
:1035C000FD000870546944F4804454615C0726D5BA
:1035D000154C22780132D2B2C82A227003D923F0C6
:1035E00006030B7010BD40F0010008700F220FE0C1
:1035F000580710D5926812F0400F4FF00F0204D018
:1036000043F002030B70094B03E043F001030B701E
:10361000074B1A7010BD536943F48043536110BDCA
:1036200065020020000C0140640200205E020020C0
:103630005F02002010B526490B7803F0040202F067
:10364000FF00002A43D1234A1278012A3FD0072ADB
:103650003DD0214A926812F0800F204A02D014789F
:103660003CB102E0107820B9012010701C4A3220D1
:1036700010701C072BD4184A9068400610D492682A
:1036800012060DD59C0703D523F002030B7007E04B
:10369000D80705D443F001030B70124B0F221A70A8
:1036A0000D4B9A68920612D49B681C060FD40B78B7
:1036B000074AD80703D523F00103137010BD9907FB
:1036C00005D443F002031370074B0F221A7010BD8C
:1036D00065020020EC000020000C0140E501002004
:1036E000460200205F0200205E020020094B1B788A
:1036F000DA0701D5084A02E09B0709D5074A137883
:103700000BB1013B03E0064A137843F080031370CA
:10371000704700BF650200205F0200205E020020AB
:10372000E8010020044B1A7802F07F021A701A7820
:1037300002F0BF021A7070471F02002070B56C4B78
:103740001B7813F0040F6B4B1A7800F0C88042F01E
:1037500080021A701A7802F0400202F0FF00002A7C
:1037600040F0C4801A7812F0200F634A16D06349E3
:103770001288098891420FD21978614C01F0DF015B
:1037800019701921B2FBF1F121805E490A801A7883
:1037900042F040021A709FE01A78A0E0197801F018
:1037A000100101F0FF00002900F08180197841F03C
:1037B00080011970197801F0BF011970197801F0B2
:1037C000040101F0FF0000293DD04F494B48B1F9F9
:1037D0000010032916DC4D4902240C70197801F001
:1037E000080101F0FF0469B90188464D29801925B7
:1037F000B1FBF5F1424D298045490C80197841F023
:103800000801197001881288023191426EDB197823
:103810003E4801F0EF0119703A490A800021017019
:103820003B4801801921B2FBF1F235490A801A7830
:1038300042F040021A701A7802F0FB021A701A78ED
:1038400002F0F70251E01488324A1288A24205D9E8
:103850002C4A14802D4A10702D4A10802E4A12785E
:10386000032A43D9254A08261588274AB2F90010A9
:10387000282251430A22624302F57A60C4F57A6233
:1038800092FBF6F290FBF2F212B291FBF2F212B25C
:103890002A4494422ADC1B4A022115801B4A1170DB
:1038A0001B4A002111801A7842F004021DE01349DE
:1038B00012880D88134CAA4214491A7806D242F095
:1038C00020021A7008700A23238070BD42F0100293
:1038D0001A701E2325800B700D4B188070BD02F0EE
:1038E0007F021A701A7802F0BF021A7070BD00BF12
:1038F000FC0100201F02002018020020A60000206A
:10390000E60100203E01002042010020400000208E
:103910000802002048020020C8000020094A13784D
:1039200003F0FB031370084B00221A70074A137848
:1039300023F020031370064AD36823F40043D360B6
:10394000704700BFFC0100201F020020DF000020A4
:10395000000C01400C4A1388022B13D9002313805A
:103960000A4A0B4913700B4A13700B4A13700A78FA
:1039700042F040020A70094A1370094A137823F092
:1039800020031370704700BF08020020EC000020E5
:10399000A8000020BE000020B50000201F0200206B
:1039A000DF00002004490B78DBB25A1CD2B20A7047
:1039B000024AD054704700BFE400002045010020B7
:1039C0002DE9F041234D244BA84600261E70FF2010
:1039D00001236B70FFF7E6FF6878FFF7E3FFA87835
:1039E000FFF7E0FFE878FFF7DDFFAB786C781C4469
:1039F000EB781C4404F0FF04EB78F7B2BB420CD91F
:103A0000474438790444FFF7CDFF3879E4B2FF2802
:103A100001D1FFF7C7FF0136EEE72046FFF7C2FFEF
:103A20000E4B00220E491A700A885206FCD51A78ED
:103A30000B48D2B2511CC9B219700A4B995CFEF7FF
:103A400043FABDE8F041012240F227710448FEF735
:103A500023BA00BF4C000020E400002040010020F9
:103A60000038014045010020F8B5B2494A780C46BB
:103A7000012A40F0AD848B782D2B00F0528232D891
:103A80000D2B00F0458116D8072B00F0F38008D8E5
:103A9000022B78D0032B00F0C380012B40F09084E0
:103AA00055E0092B00F02781C0F017810B2B00F0A7
:103AB0002F8100F085BC142B00F0CC8109D8102B8D
:103AC00000F0A281112B00F0AF810F2B40F0788421
:103AD0008BE1262B00F066832C2B00F0FC81252B3C
:103AE00040F06E84CEE23E2B00F0E08217D8382BF7
:103AF00000F0648209D8342B00F03B82372B00F0B1
:103B00004A82332B40F05C8424E23C2B00F06E822E
:103B100000F27682392B00F05E8200F051BC522B0D
:103B200000F0D78309D8452B00F09883512B00F083
:103B3000BA833F2B40F044843EE3622B00F0E183E4
:103B4000632B00F01B84552B40F03A84CBE3CA78FA
:103B5000784B22B10123E370032300F034BC0C2125
:103B6000D970032119719A720121DA72724A59715E
:103B700099711F21D97112690A2119721221597282
:103B8000DA6000F021BCCB78012B09D16B496C4B7A
:103B9000CA6802F4E0621343CB60BFF34F8FFEE7C5
:103BA000002BD7D1674A0123CB700B7111780729FD
:103BB00006D1614B64481D8B0580D88A634B188001
:103BC00063480229037808BF624923F02003037089
:103BD000614818BF6149037823F008030370604807
:103BE0004FF0000303705F4803705F4803705F4845
:103BF0004FF00F0303705E48037015BFCB680B785E
:103C000043F0400343F0010314BFCB600B7000236B
:103C10001370584A1380584A1380584A1370B4E1FD
:103C2000CB78002B96D10423CB70554B1B888B800F
:103C3000544B1B78CB71544B9B689D0607D4444B67
:103C40001B7813F0200F14BF0323002300E003238D
:103C5000434A117808061178127848BF43F01003E0
:103C6000890748BF43F02003520648BF43F0400392
:103C7000A371A9E3CB78002B7FF46CAF3648344DA9
:103C8000017841F0040101702878404920F02000BB
:103C90000B702870324933480B7003703248037040
:103CA000087800F0EF000870087800F0DF00087076
:103CB00024490B7033490B702E490B802E490B8021
:103CC0002E490B7032490B7843F040030B702349A7
:103CD000CB6843F04003CB60E2E2CB78002B7FF46B
:103CE00039AF1D4A137823F0050343F00203137024
:103CF0000F221F4B77E0CB78002B7FF42BAF0223F2
:103D0000CB70224B1B780B71134B1B784B715BE311
:103D1000E178084B01297FF41DAF1A79012A03D9F4
:103D20000422D9701A714FE31A49AABB0B7803F029
:103D3000FB0340E04C0000202402002000ED00E0E6
:103D40000400FA05EC000020660200206202002058
:103D5000DF000020C30000206502002000080140B1
:103D60001F020020E8010020410200205F02002025
:103D70005E020020E60100204802002040000020F2
:103D8000A6000020B5000020000C014064020020C5
:103D9000A8000020FC0100209E4B1A889E4B1A8030
:103DA0005A809A80DA801A815A819C4B64221A8048
:103DB0000B7843F004030B70994B00221A70994B57
:103DC0001A7802F0BF021A701A7802F0EF021A7025
:103DD0001A7802F0DF021A701A7802F0FB021A70E9
:103DE0001A7802F0F7021A70EEE2CB78002B7FF41B
:103DF000B1AE8D4A07218D48D170E218195C0133AC
:103E0000072B1171F9D1DFE2CB78072B7FF4A2AE3B
:103E1000864A0023E1180979834D99540133072B11
:103E2000F8D1FEF71DFC68E2CB78012B7FF492AE4F
:103E30000B79012B04D17B4A137803F0FE0305E0D4
:103E4000022B04D1774A137843F00103137000F07A
:103E500011FEB9E2CB78012B7FF47CAE0B793BB934
:103E600073490A7802F0FB020A70724A137019E073
:103E7000012B17D1674B1A88674B1A805A809A809A
:103E8000DA801A815A81654B64221A806A4B4FF49A
:103E900048721A80664A137843F004031370654B26
:103EA00006221A705E4B00221A705E4B1A7802F0DE
:103EB000BF021A701A7802F0EF021A701A7802F034
:103EC000DF021A701A7802F0FB021A701A7802F0F8
:103ED000F7021A70BFE1CB78002B7FF43BAE0123D1
:103EE000504ACB700B7100231370544A544913701D
:103EF000544A1370494A1380534A1380484A137036
:103F00000A7842F040020A704A4A072111704F496C
:103F10000A7842F020020A704D4A13704D4A13800D
:103F200052E2CB78002B7FF415AE0A23CB704A4BBC
:103F30001B888B80494B1B88CB80494B1B880B818E
:103F4000484B1B884B81484B1B780B73474B1B78A6
:103F50004B7339E2CB78002B7FF4FCAD324A1A2147
:103F60004348D170E218195C01331A2B1171F9D151
:103F70002AE2CB781A2B7FF4EDAD3D4A0023E118FD
:103F80000979995401331A2BF9D12D4A137843F04A
:103F90004003137018E2CB78002B7FF4DBAD40F6C2
:103FA000E4400623334DCB7000235A5BE1184243B3
:103FB0000233120B062B8A80F7D105E2CB78002B57
:103FC0007FF4C8AD0423CB70224B1B888B801E4B23
:103FD0001B88CB80F8E1CA78134B002A7FF4BAAD76
:103FE0000222DA70244A12889A80EDE1CB78002B05
:103FF0007FF4B0AD0223CB70204B1B888B80E3E1B4
:10400000CB78002B7FF4A6AD1D4A137843F0040350
:10401000137020E1A60000204C020020E6010020E1
:10402000400000201F0200204C0000200002002061
:10403000FC010020EC00002018020020E801002014
:10404000A80000204102002048020020DF000020DC
:10405000BE00002008020020600200205C02002058
:1040600062020020660200203C0000203D0000208B
:1040700024020020EC0100201C0200203801002056
:10408000C3000020A64A137843F020031370A54A0A
:10409000137843F008011170A34989684F0605D4CD
:1040A00043F009031370A14B0F221A70E378482BD9
:1040B0007FF450AD9E4A0023E118097999540133E9
:1040C000482B9B49F8D14878954B10F0800F03D0CE
:1040D0001A7862F07F0204E0460603D51A7842F0AF
:1040E00040021A7000F03F0048701878904A00F0C3
:1040F000200000F0FF03B0B14FF6FF758D48968A9F
:1041000005803C20508036B11589108A281A90FB12
:10411000F6F0508200E05682088A002208831E20B2
:104120008A8248830A84844802260670834A844827
:10413000002515700570834D40262E70824FEBB11F
:104140003B88824982480B800021018081480170B0
:104150002321B3FBF1F380490B80137803F0DF03D5
:104160001370137803F0EF031370137803F0F70361
:104170001370137803F0FB03137068E01D460E887C
:10418000B7F800E0764509D2632E07D90233DBB2D7
:10419000122B05D031F823600125F3E7002DCFD095
:1041A0000370CDE75E4A137843F0200313705D4A35
:1041B000137843F008031370E378482B7FF4CAACFC
:1041C0005B490022A3181B7953540132482A584BEB
:1041D000F8D15878524910F0800F03D00A7862F075
:1041E0007F0204E0450603D50A7842F040020A70D7
:1041F000097800F03F0089064D4A587016D54FF6F1
:10420000FF704C49958A08803C21518035B1108956
:10421000118A411A91FBF5F1518200E05582198A09
:10422000002219831E219A8259831A84434B1A78DB
:1042300002F0FB021A701B7803F0400303F0FF0248
:104240002BB9414B1988414B1980414B1A80FEF71D
:104250002FF9FEF7A7FA0123E370B4E0CB78002B27
:104260007FF478AC36490B70344B197801F0DF01DC
:104270001970197801F0EF011970197801F0FB013C
:104280001970197801F0F701197034490B7803F0AF
:10429000FB030B70304B64211980274B05211970EB
:1042A000E270227190E0CB78002B7FF453AC0923AD
:1042B000CB702B4B1B88CB802A4B1B780B71264B6A
:1042C0001B880B81284B1B884B81284B1B888B81BB
:1042D0007AE0CB78002B7FF43DAC0423CB70244BE9
:1042E0001B684B6070E0CB78224D042B7FF432AC1E
:1042F0006A68214B1A61FEF7D9F80123EB702B7124
:1043000062E0CB78002B7FF425AC48220848CA70C5
:10431000E218195C0133482B1171F9D154E000BF48
:10432000DF00002065020020000C01405F02002039
:10433000EE00002014000020EC0000201F020020EE
:10434000BE000020B5000020A60000203E01002095
:104350000802002040000020E6010020C3000020E9
:104360004201002016000020E00000200E02002084
:10437000B80000204C00002024020020CB78002B45
:104380007FF4E8AB0323CB70124B1B78022B0B712D
:104390000AD1114B1B781A0642BF104A82211171B3
:1043A0005B0644BF422323710D4B0C4A1B7863719B
:1043B0000C4B1B7813F0010318BF0123937103E02A
:1043C0000123E37002232371FFF7FAFA064B1C6006
:1043D000F8BD00BFEC000020DF0000204C000020F2
:1043E000580200201F020020440000202DE9F04761
:1043F000234B00201E7802463146224B224CB3F854
:104400000080224BDFF888E01F8820603C254FF0B9
:10441000030C11292FD84FEA410A11F0010F3EF881
:104420001A3006D0B14205FB032220D1C8EB0202AC
:104430001DE0632B1FD90AF10100B1423EF8109034
:1044400005D1BB4201D2FB1A08E0DB1B0BE0AAF14D
:10445000040A3EF81A00834204D2C31A6B4393FB4A
:10446000FCF303E01B1A6B4393FBF9F31A4401318D
:10447000C9B20120CDE700B12260BDE8F08700BFDE
:10448000BE00002008020020B8000020A600002086
:10449000EE00002030B5264B26481A78264942F017
:1044A00080021A701A7842F040021A70234B1A8860
:1044B000234B1A80234B1A80234B1B78052B15D0D6
:1044C00003880C881433A34210DB204B204C1B784C
:1044D00001335B0034F81350954207D9013334F8A7
:1044E00013301C4C03EB83035B0023800B88048890
:1044F00019499C4202D20B785B0718D54FF6FF751D
:10450000124C23780133DBB22370144C2580002435
:104510000480087800F0FB0008700D4931F8233062
:104520009A423FBF0F22B3FBF2F30A4A138030BD19
:104530001F02002008020020FE0100203C01002094
:104540003E01002048020020EC000020BE000020B8
:10455000EE000020E6010020C3000020140000202F
:1045600070B55F4B5F491A7842F080021A701A7872
:1045700042F040021A705C4B5C4A18885C4B188011
:104580005C4B18805C4B1B78052B15D05B4B14885B
:104590001B881433A3420FDB0B78594C01335B00AB
:1045A00034F81350854207D9013334F81330554C91
:1045B00003EB83035B0023801288EAB90B78012B9D
:1045C0000BD1514B9B689C0616D4504A137843F08C
:1045D000020313700F224E4B0CE0072B0CD14A4BF9
:1045E0009B685B0608D4494A137843F001031370B3
:1045F000484B0F221A7070BD404C238825469A42C2
:1046000003D9454C2678760726D53F4B9A68920603
:1046100002D40A78012AD8D09B685B0602D40B78B2
:10462000072BE0D00B783D4A0133DBB20B704FF61D
:10463000FF711180384900222A800A7802F0FB02BB
:104640000A702F4A32F82330984247D20F22B3FB28
:10465000F2F32C4A138070BD0978012922D12F482A
:104660000188994215D00A21B2FBF1F2B3FBF2F1B5
:1046700002FB113292B2032A0BD124490A78960622
:1046800007D442F020020A70254A03801188254A87
:1046900011801D4B9B689D0620D5237843F00403B1
:1046A000237070BD072919D11C480188994215D083
:1046B0000A21B2FBF1F2B3FBF2F102FB113292B22A
:1046C000032A0BD111490A78D40607D442F010020C
:1046D0000A70154A03801188124A118070BD00BF0C
:1046E0001F020020BE0000203C010020FE0100202F
:1046F0003E01002048020020EC00002008020020BB
:10470000EE000020E6010020000C014065020020C0
:104710005E0200205F020020C30000201400002081
:1047200066020020180000206202002010B5324B03
:1047300032491B78324A13F0200F324B24D03248D2
:10474000806884060AD40C881088844206D92F48D1
:10475000007818B9187800F07F0002E0187840F06F
:10476000800018701878128800F0BF00098818704F
:10477000501D814203DD2548007800283AD00131E0
:104780008A42234911DD0DE01878098840F0800045
:10479000187018781288013100F0BF00914218702B
:1047A0001B4902DA0878400724D5184C19480280C2
:1047B00020780130207018480024048017480280B7
:1047C0001920B2FBF0F21648B0F900409442C8BF7D
:1047D00002801A7802F0FB021A701A7802F0F702CF
:1047E0001A700B780F4A03F0FB030B70137843F039
:1047F0004003137010BD00BFDF000020A6000020A2
:104800003C0100201F020020000C0140BE000020DF
:10481000C30000203E0100200802002048020020C2
:10482000E6010020A800002070B5294B294C1B7818
:10483000294813F0200F294A294B22D02949498AB7
:10484000F9B1294D2E78042E2E461AD17D29274DF7
:104850008CBF832149422970197841F08001197079
:10486000197801F0BF01197021880488881C8442DE
:1048700002DD107844072AD51D48018005203070DC
:1048800015E0197801F07F011970197801F0BF0166
:10489000197021880488881C844202DD1078400742
:1048A00015D51348104C0180207801302070114834
:1048B000002404801E20B1FBF0F10F48018019781C
:1048C00001F0FB011970137803F0FB03137070BD46
:1048D000DF0000203C010020A6000020C3000020D3
:1048E0001F020020EE000020BE000020400000203B
:1048F0003E01002008020020E60100202DE9F041E1
:10490000DFF86C8198F80030464613F0010F40F054
:104910008E80484D484C2B78484F43F0400323701D
:10492000FFF764FD2A784648510012F0010F30F875
:104930001130864618D03978424801F0200101F044
:10494000FF0409B1032A02D0C3EB03139B000380C9
:104950003D4B00221A701CB1BDE8F041FFF700BECC
:10496000BDE8F041FFF796BD632B01D9112A24D988
:10497000202323703378002003F07F0333703378D3
:1049800003F0BF033370314B18803B7813F0200FD6
:104990002F4B14BF0320042018702E48012A0378DF
:1049A00043F04003037042D904393EF811302A4ADB
:1049B00013802A4A1380BDE8F081013130F81100DC
:1049C00027490B8098F8001011F0040F1E4905D0FC
:1049D00091F90000022804DD022001E000B9012065
:1049E0000870397889061AD5042A03D1BDE8F04148
:1049F000FFF71ABF062A03D107232B70BDE8F08109
:104A00006AB9184A9268520609D4174917480A78B1
:104A10000F2422F0020242F0010204700A700E4AD2
:104A200012889A42E2D8BDE8F041FFF77FBEBDE8A8
:104A3000F08100BFBE000020B5000020DF00002094
:104A4000EE000020FE0100204000002008020020AF
:104A5000EC000020A80000203E01002048020020B9
:104A60003C010020000C0140650200205F02002094
:104A70001F0200200E4B00221A800E4B1A7812F0F3
:104A8000010F1A780BD002F0FE021A701A7802F0A9
:104A9000FB021A701A7802F0F7021A70704742F09F
:104AA00001021A70044B1A88044B1A80704700BF29
:104AB000380100201F020020A60000204A0200202A
:104AC000144B1A88B2F5616F1A46134B03D8134979
:104AD0000978890612D5197801F07F0119701978C3
:104AE00001F0BF011970002313800D4B03221A70CF
:104AF0000C4A137843F04003137070471A7842F061
:104B000080021A701A7842F040021A70064B202276
:104B10001A707047080200201F020020DF000020EA
:104B2000EC000020A8000020B500002010B5424C89
:104B30002378062B7FD8DFE803F00412272E3542B6
:104B40004F00FE20FDF7A4FB3C4B1A883C4B1A801B
:104B50003C4B00221A8023780133DBB21FE040F285
:104B60001A42394B1A80394B1B7813F0040F384B1B
:104B700005D093F90020022A03DD022200E046223C
:104B80001A70FFF7D3FD23E0324B4FF416721A80F0
:104B9000FFF780FC1CE0304BFE22DA8104232370F7
:104BA0002E4A47E02E4B9B689A0603D52A4BDB8999
:104BB0000A2B0DD8234B00221A80052307E0284B2F
:104BC0009B689B0604D51F4B00221A800623237086
:104BD0002278224B1A7010BD1F4AD389F82B9CBF34
:104BE0000533D381194B1A7802F07F021A701A78B4
:104BF00002F0BF021A701A7802F0DF021A701A78F7
:104C000002F0EF021A701A7802F0FB021A701A789A
:104C100002F0F7021A70134B03221A70094B00229C
:104C20001A80072323700D4B20221A700E4A137826
:104C300043F04003137010BDBE000020A60000200A
:104C40003E010020080200203C0100201F0200203D
:104C500040000020FE01002024020020B5000020BA
:104C600000080140EC000020A800002038B57E4C70
:104C70002378072B00F2E980DFE803F0040B1D2CFA
:104C80003B5C82A4794B9B6899062AD5012323704B
:104C90001BE0774B1B88002B40F0E280754A1380A5
:104CA000754A02232370137843F001031370734B8A
:104CB0000F221A70D4E06D4B9B685A0640F1D080E9
:104CC000032323706E4B00221A80694B4FF47A72D3
:104CD0001A80C5E0664B1B88002B40F0C18004237E
:104CE0002370654A137843F0020313700F22654B5B
:104CF000DFE75E4B9B689B0640F1B2800523624A6A
:104D0000237000231370614A1370614A1370614A63
:104D10001370614A1370574B0C221B88B3FBF2F3DC
:104D20005E4A1380564B11221B88B3FBF2F35C4A98
:104D30001380CAE74D4B4E4A9B6813F0400F05D0D5
:104D4000062323704FF47A73138089E01388002BB5
:104D500040F086804E4B1978474B61B94A4801783C
:104D60000131017040F6B83111801A7842F010021A
:104D70001A704A4B23E01A7842F001021A7096E743
:104D80003A4B9B6813F0200F394B04D00722227056
:104D90004FF47A729CE71A88002A61D13D4A127852
:104DA000002A9ED139490A7801320A7040F6B83299
:104DB0001A80314A137843F020031370384B1A8855
:104DC000384B85E7344A13780133DBB2032B137079
:104DD0000FD9334A344B12881A83304A1288DA8248
:104DE000FDF764FB40F6B832214B1A80237801337B
:104DF00035E025490B78A3F10902022A234A07D896
:104E00001378093B022BE4D9214B0121197008E0EA
:104E1000224805886B430A25B3FBF5F30380002382
:104E20000B701378A3F10902022A09D91C4A1188D0
:104E30004B430A21B3FBF1F313800022134B01E033
:104E4000144B01221A70052309E0184A184900235F
:104E500013700A7822F020020A70074A1370237038
:104E60002278144B1A7038BDBE000020000C01409F
:104E70001A00002060020020650200205F0200206E
:104E80005C0200205E0200203C0000203D0000206B
:104E90003B0000203E0000203A000020620200207B
:104EA000660200201800002024020020EC000020F0
:104EB000DF000020B50000207047FEE7FEE7FEE7B8
:104EC000FEE7704770477047234A13680133B3F514
:104ED0007A7F136006D300231360204A137843F0CF
:104EE0008003137041F288311D4A138801339BB24D
:104EF0008B42138006D900231380184A137843F09D
:104F000008031370174A13780133DBB2032B81BFF8
:104F100000231370144A137888BF43F020031370E2
:104F2000124A13880BB1013B1380114A13880BB14D
:104F3000013B13800F4B1B78072B0CD10E4B1B78BA
:104F4000022B02D0042B02D070470C4A00E00C4A1E
:104F50001388013313807047E8000020A800002068
:104F60004202002039000020C30000201800002069
:104F70001A000020EC000020BE000020600200208B
:104F80005C02002008B50120FCF70CFF20B1BDE851
:104F900008400120FCF716BF08BD000008B502203C
:104FA000FCF76AFDB0B10220FCF774FD0A4B1A78D9
:104FB00092060FD51A78002102F0DF021A70074A14
:104FC000117007490A7842F004020A701A7842F018
:104FD00010021A7008BD00BFC30000203900002075
:104FE000A800002008B50120FCF746FD002833D0BA
:104FF0000120FCF74FFD194B1A78D2062CD51A78F0
:1050000002F0EF021A70164B1B7803F0020303F054
:10501000FF0043B1134A1378FF2B1DD013780133DF
:10502000DBB2137008BD104A13780133DBB2282BB2
:10503000137011D910700D4A13780133DBB20A2BAB
:10504000137009D910700A4AD36823F40043D3605F
:10505000BDE80840FDF724B908BD00BFC30000202B
:105060001F0200200C02002040020020C700002088
:10507000000C014010B5084C4FF408712046FCF7B5
:10508000EEFB10212046FCF7E7FB044A137843F0BF
:105090008003137010BD00BF00240140FC010020FC
:1050A00070B5424C40F225512046FCF715FF002810
:1050B0005AD02046FCF70CFF23881A0754D42388C3
:1050C0009B0751D43A4BC0B21A783A4912F0040FF8
:1050D000394A12D0FF280AD1147834B10C68013C47
:1050E0000C601478013CE4B214701C7810E0334C6E
:1050F0002070334C0C600124F6E7304DFF282C78EB
:105100000444E4B22C701C7802D144F0040401E0A1
:1051100004F0FB041C700C68651C0D602070147892
:105120000134E4B24F2C147082BF234C002525704B
:105130001478042C18D9204C2678224CE5780435B4
:10514000AE42254610DD1D4C0D602478241AE4B2D1
:10515000A04202BF187840F00800187000201070BC
:105160001A7802F0FB021A7040F227710F48FCF720
:10517000B3FED0B11049144B0A781B789A4208D379
:1051800000220A70094840F22771BDE87040FCF720
:1051900083BE0B780548DBB25A1CD2B20A700B4AA8
:1051A000BDE87040D15CFCF78FBE70BD0038014097
:1051B0001E0200204400002040010020BF0000200B
:1051C0004D0000204C000020E4000020450100209C
:1051D000304B82B01A6842F001021A6059682E4AB8
:1051E0000A405A601A6822F0847222F480321A60EF
:1051F0001A6822F480221A605A6822F4FE025A6069
:105200004FF41F029A600022DA62009201921A683B
:1052100042F480321A601A6802F400320192009A55
:1052200001320092019A1AB9009AB2F5A06FF2D138
:105230001A6812F4003218BF01220192019A012A61
:1052400004D0164A164B9A6002B070475A685A60EA
:105250005A685A605A685A605A6822F47C125A6036
:105260005A6842F410225A601A6842F080721A603A
:105270001968084A8901FBD5516821F00301516082
:10528000516841F0020151605A6802F00C02082A8C
:10529000FAD1D6E7001002400000FFF80014000821
:1052A00000ED00E040F24C43984228BF1846024B04
:1052B00033F81000704700BFF05300084BF23F0373
:1052C0009842F0B528D840F24C42164E00218C1876
:1052D000641036F81470A3B2B8420CD25A1E92B2BF
:1052E00036F81250A84214D93D44B0EB650FD4BF34
:1052F00010461846F0BD12D9591C89B236F8114033
:10530000A04206D23C44B0EB640FCCBF084618461E
:10531000F0BD9142DBD902E040F24C40F0BD1846AE
:10532000F0BD00BFF05300080E4B70B51E460E4C8A
:105330000025E41AA410A54204D056F82530984759
:105340000135F8E700F006FD084B094C1E46E41A4B
:10535000A4100025A54204D056F825309847013501
:10536000F8E770BD6C5D00086C5D00086C5D0008BE
:10537000705D0008320032003200320032002C0032
:10538000FC03FA0000000000410041004100410020
:105390004100D200A406FE0000000000230023000C
:1053A0002300230023000100F401B40000000000EA
:1053B00063000100000000001A043C00FC03FC0331
:1053C0001F1F1C1F1E1F1E1F1F1E1F1E1F00000051
:1053D000253700081D390008FD4800085539000828
:1053E000C14A00082D4B00083D3700086D4C0008ED
:1053F000000027004F0077009E00C600EE00150158
:105400003D0165018D01B501DD0105022D02550249
:105410007D02A502CE02F6021E0346036F03970328
:10542000C003E8031104390462048B04B304DC04F0
:1054300005052E0556057F05A805D105FA052306A5
:105440004C0675069E06C706F006190742076B074D
:105450009507BE07E70710083A0863088C08B608E6
:10546000DF08080932095B098409AE09D709010A76
:105470002A0A540A7D0AA70AD00AFA0A230B4D0BFE
:10548000760BA00BC90BF30B1C0C460C700C990C83
:10549000C30CEC0C160D3F0D690D920DBC0DE50D06
:1054A0000F0E380E620E8B0EB50EDE0E080F310F8A
:1054B0005B0F840FAD0FD70F00102A1053107C1014
:1054C000A610CF10F81021114B1174119D11C611A7
:1054D000EF11191242126B129412BD12E6120F1341
:1054E000381361138A13B313DC1304142D145614E8
:1054F0007F14A814D014F91422154A1573159C159D
:10550000C415ED1515163E1667168F16B716E0165C
:105510000817311759178117AA17D217FA17231826
:105520004B1873189B18C318EC1814193C196419FC
:105530008C19B419DC19041A2D1A551A7D1AA51ADA
:10554000CD1AF51A1D1B451B6D1B941BBC1BE41BC0
:105550000C1C341C5C1C841CAC1CD41CFC1C241DAA
:105560004C1D741D9B1DC31DEB1D131E3B1E631E96
:105570008B1EB31EDB1E031F2B1F531F7B1FA31F7E
:10558000CA1FF21F1A2042206A209220BA20E2206D
:105590000A2133215B218321AB21D321FB2123224B
:1055A0004B2273229C22C422EC2214233C23652329
:1055B0008D23B523DD2306242E2456247F24A724FF
:1055C000CF24F8242025492571259A25C225EB25CD
:1055D00013263C2664268D26B526DE2607272F2790
:1055E00058278127A927D227FB2724284C2875284C
:1055F0009E28C728F028182941296A299329BC29FF
:10560000E5290E2A372A602A892AB22ADB2A042BA6
:105610002D2B562B7F2BA82BD12BFB2B242C4D2C49
:10562000762C9F2CC92CF22C1B2D442D6E2D972DE2
:10563000C02DE92D132E3C2E652E8F2EB82EE12E77
:105640000B2F342F5E2F872FB12FDA2F03302D3001
:1056500056308030A930D330FC302631503179318A
:10566000A331CC31F6311F32493273329C32C6320B
:10567000F032193343336D339633C033EA33133486
:105680003D3467349134BA34E4340E3538356135FD
:105690008B35B535DF35093632365C368636B03671
:1056A000DA3604372E3757378137AB37D537FF37E0
:1056B000293853387D38A738D138FB3825394F3948
:1056C0007939A339CD39F739213A4B3A753A9F3AAE
:1056D000C93AF33A1D3B473B713B9B3BC53BEF3B14
:1056E000193C433C6D3C973CC23CEC3C163D403D74
:1056F0006A3D943DBE3DE93D133E3D3E673E913ED1
:10570000BB3EE63E103F3A3F643F8E3FB93FE33F2A
:105710000D40374062408C40B640E0400B4135417F
:105720005F418A41B441DE41084233425D428742D3
:10573000B242DC42064331435B438543B043DA4324
:1057400005442F4459448444AE44D84403452D4570
:1057500058458245AD45D74501462C4656468146BB
:10576000AB46D64600472A4755477F47AA47D44706
:10577000FF47294854487E48A948D348FE4828494D
:1057800053497D49A849D249FD49274A524A7C4A92
:10579000A74AD24AFC4A274B514B7C4BA64BD14BD4
:1057A000FB4B264C514C7B4CA64CD04CFB4C264D15
:1057B000504D7B4DA54DD04DFA4D254E504E7A4E55
:1057C000A54ECF4EFA4E254F4F4F7A4FA54FCF4F94
:1057D000FA4F24504F507A50A450CF50FA502451D1
:1057E0004F517951A451CF51F95124524F5279520E
:1057F000A452CF52F95224534E537953A453CE534B
:10580000F95324544E547954A454CE54F954245585
:105810004E557955A455CE55F95524564E567956C0
:10582000A356CE56F95623574E577957A357CE57FE
:10583000F95723584E587958A358CE58F858235939
:105840004E597859A359CE59F859235A4D5A785A76
:10585000A35ACD5AF85A235B4D5B785BA25BCD5BB4
:10586000F85B225C4D5C775CA25CCD5CF75C225DF2
:105870004C5D775DA25DCC5DF75D215E4C5E765E32
:10588000A15ECB5EF65E215F4B5F765FA05FCB5F74
:10589000F55F20604A6075609F60CA60F4601F61B8
:1058A000496174619E61C961F3611E6248627362FD
:1058B0009D62C862F2621D63476372639C63C76343
:1058C000F1631B64466470649B64C564F0641A658C
:1058D00044656F659965C465EE65186643666D66D7
:1058E0009766C266EC66166741676B679567C06727
:1058F000EA6714683F6869689368BE68E868126977
:105900003C6967699169BB69E569106A3A6A646ACA
:105910008E6AB86AE36A0D6B376B616B8B6BB66B23
:10592000E06B0A6C346C5E6C886CB26CDD6C076D7D
:10593000316D5B6D856DAF6DD96D036E2D6E576EDC
:10594000816EAC6ED66E006F2A6F546F7E6FA86F3B
:10595000D26FFC6F267050707A70A370CD70F770A4
:1059600021714B7175719F71C971F3711D7247720D
:1059700071729A72C472EE72187342736C7395737B
:10598000BF73E97313743D7466749074BA74E474ED
:105990000D75377561758A75B475DE750876317663
:1059A0005B768576AE76D87602772B7755777E77DD
:1059B000A877D277FB7725784E787878A178CB785E
:1059C000F4781E79477971799A79C479ED79177AE3
:1059D000407A6A7A937ABD7AE67A107B397B627B69
:1059E0008C7BB57BDE7B087C317C5A7C847CAD7CF7
:1059F000D67C007D297D527D7C7DA57DCE7DF77D89
:105A0000217E4A7E737E9C7EC57EEF7E187F417F1D
:105A10006A7F937FBC7FE67F0F80388061808A80B9
:105A2000B380DC8005812E8157818081A981D2815C
:105A3000FB8124824D8276829F82C882F1821A8302
:105A400043836C839583BE83E783108438846184A9
:105A50008A84B384DC8405852D8556857F85A88559
:105A6000D185F98522864B8674869C86C586EE860E
:105A700016873F8768879087B987E2870A883388C7
:105A80005C888488AD88D588FE8826894F89788986
:105A9000A089C989F1891A8A428A6B8A938ABC8A49
:105AA000E48A0C8B358B5D8B868BAE8BD68BFF8B14
:105AB000278C508C788CA08CC98CF18C198D428DE0
:105AC0006A8D928DBA8DE38D0B8E338E5B8E848EB4
:105AD000AC8ED48EFC8E248F4D8F758F9D8FC58F8D
:105AE000ED8F15903D9065908E90B690DE9006916A
:105AF0002E9156917E91A691CE91F6911E9246924C
:105B00006E929692BE92E6920E9336935D93859333
:105B1000AD93D593FD9325944D9475949C94C49422
:105B2000EC9414953C9563958B95B395DB95029613
:105B30002A9652967A96A196C996F196189740970A
:105B400068978F97B797DE9706982E9855987D9807
:105B5000A498CC98F3981B9943996A999299B9990A
:105B6000E199089A2F9A579A7E9AA69ACD9AF59A11
:105B70001C9B439B6B9B929BBA9BE19B089C309C1C
:105B8000579C7E9CA59CCD9CF49C1B9D439D6A9D2F
:105B9000919DB89DDF9D079E2E9E559E7C9EA39E47
:105BA000CB9EF29E199F409F679F8E9FB59FDC9F63
:105BB00003A02AA052A079A0A0A0C7A0EEA015A182
:105BC0003CA163A18AA1B1A1D7A1FEA125A24CA2AB
:105BD00073A29AA2C1A2E8A20FA335A35CA383A3D8
:105BE000AAA3D1A3F8A31EA445A46CA493A4B9A40A
:105BF000E0A407A52EA554A57BA5A2A5C8A5EFA541
:105C000016A63CA663A689A6B0A6D7A6FDA624A77D
:105C10004AA771A797A7BEA7E4A70BA831A858A8C1
:105C20007EA8A5A8CBA8F2A818A93FA965A98BA909
:105C3000B2A9D8A9FEA925AA4BAA71AA98AABEAA58
:105C4000E4AA0BAB31AB57AB7DABA4ABCAABF0ABAB
:105C500016AC3CAC62AC89ACAFACD5ACFBAC21AD06
:105C600047AD6DAD93ADB9ADE0AD06AE2CAE52AE65
:105C700078AE9EAEC4AEEAAE10AF35AF5BAF81AFCB
:105C8000A7AFCDAFF3AF19B03FB065B08AB0B0B039
:105C9000D6B0FCB022B147B16DB193B1B9B1DEB1AC
:105CA00004B22AB24FB275B29BB2C0B2E6B20CB324
:105CB00031B357B37CB3A2B3C8B3EDB313B438B4A4
:105CC0005EB483B4A9B4CEB4F4B419B53EB564B52A
:105CD00089B5AFB5D4B5F9B51FB644B669B68FB6B8
:105CE000B4B6D9B6FFB624B749B76EB793B7B9B74C
:105CF000DEB703B828B84DB872B898B8BDB8E2B8E6
:105D000007B92CB951B976B99BB9C0B9E5B90ABA86
:105D10002FBA54BA79BA9EBAC3BAE8BA0CBB31BB2F
:105D200056BB7BBBA0BBC5BBE9BB0EBC33BC58BCE0
:105D30007CBCA1BCC6BCEBBC0FBD34BD59BD7DBD98
:105D4000A2BDC6BDEBBD10BE34BE59BE7DBEA2BE57
:105D5000C6BE0000F8B500BFF8BC08BC9E46704740
:0C5D6000F8B500BFF8BC08BC9E467047B8
:045D6C00F515000821
:045D7000D115000841
:105D740002040608000000000102030401020304F7
:0C5D840006070809FFFFFE006400D007BE
:0400000508001611C8
:00000001FF
